:1000000054C06EC049C76CC06BC06AC069C068C0CC
:1000100067C066C065C04AC963C0E1C861C060C04E
:100020005FC05EC05DC00403090418037A00650068
:10003000720074006900650073002E006F0072008A
:1000400067001203650074006800650072007300A9
:100050006500780012011001FF000008C016DC05E1
:1000600000010102000109021200010100800F09D4
:100070000400000000000000626F6F746C6F616428
:10008000657200696F20007800C4098300740A005B
:100090000000007061727365206572726F7200708B
:1000A0006F727420503A2030780011241FBECFE5C3
:1000B000D4E0DEBFCDBF10E0A0E6B0E0E0EFF6E1B7
:1000C00002C005900D92A239B107D9F712E0A2E95A
:1000D000B0E001C01D92A63DB107E1F702D006CB0A
:1000E0008FCFCF93DF9378948FE028E130E00FB685
:1000F000F894A89521BD0FBE81BDA89524D034D019
:1001000088D42DD88091A600897F8093A600C0E076
:10011000D0E0A895D4D7A89593D4A8952CD0A8952D
:10012000A8958091A60081FF06C0F894E091600038
:10013000F091610009958091A60082FFEACFF894C2
:10014000FE010995E6CF0F931F9302E810E010938C
:100150008F0000938E004FD110938F0000938E007C
:1001600071D01F910F9108958DE08EBD88E391E0CD
:100170009BBD8ABD08951F93CF93DF9308B604FEFD
:1001800052C080E188BF80919200909193000196C7
:10019000909393008093920087709070892B09F55B
:1001A00000D8CDE8D1E016E08E89819FC0011124EE
:1001B0008E579F4F90938F0080938E00D093AF0007
:1001C000C093AE0085E05CD18091A7009091A8001B
:1001D000892B11F074D35DD3679622E0C030D2072B
:1001E00019F7809192009091930062E370E06ADACF
:1001F000892B41F48091A7009091A800892B11F0E0
:100200005ED347D38091920090919300845F914098
:1002100021F410929300109292008091C5028823DD
:1002200011F41092B800DF91CF911F910895E091E1
:10023000AE00F091AF000488F589E02D309709F009
:100240000995089567D00895DF93CF93CDB7DEB7B2
:1002500067970FB6F894DEBF0FBECDBF8091AB009D
:1002600081FF4FC0E091B400F091B500DE0111961E
:10027000B89780E101900D928150E1F7E091B400D0
:10028000F091B500F09780A591A5F0969C8B8B8B93
:100290008AE09DE89A8B898BCE0101969093AF00FE
:1002A0008093AE008091A7009091A8008E0F9F1FB1
:1002B00020812D3011F02A3011F4108204C03196C3
:1002C000E817F907A8F36091B4007091B500CB016D
:1002D00040E950E064D8019690938C0180938B01A3
:1002E000E091B400F091B500E80FF91F31978AE072
:1002F000808384E0C5D0E3D2CCD210928C011092DE
:100300008B0167960FB6F894DEBF0FBECDBFCF91BD
:10031000DF910895DF93CF93CDB7DEB760970FB627
:10032000F894DEBF0FBECDBFDE011196E2E6F0E02D
:1003300080E101900D928150E1F7CE01019660E0DD
:1003400070E044E251E028D2FC01009721F08AE0FD
:100350009DE8918B808B60960FB6F894DEBF0FBE40
:10036000CDBFCF91DF9108959C0141505040460F81
:10037000571FFB010EC0708160E08181DB01A80F77
:10038000B11D2A0F3B1F2A173B0710F42F5F3F4F69
:100390003296E417F50778F3E417F50749F49081EE
:1003A00080E0280F391F2817390710F42F5F3F4FBF
:1003B000C90108950F931F931091DB0000E0909105
:1003C000DC00090F111D9801280F311DC9016FEDC7
:1003D00070E040E250E0C8DF6FEF70E0A801C4DFDA
:1003E000009719F42FEF3FEF02C0382F292FC901D2
:1003F0001F910F91089580E094E09093AD00809359
:10040000AC000895DC01FB0107C09C918081981726
:10041000F1F41196319648504830B8F74423C9F0AA
:100420008081282F30E08C9190E02827392768E0E0
:1004300070E0CB01841B9109F90102C0F595E795A5
:100440008A95E2F7E0FD03C0415099F702C080E0D1
:10045000089581E00895AC01FB01161617067CF49F
:1004600060938B01F0938C012091A9003091AA0038
:100470008217930721F0C901BA01AF011AD9089573
:100480001F93CF93DF93843009F40DC143E151E012
:100490005093B5004093B4005093AA004093A90034
:1004A000853019F5E091AE00F091AF008089918917
:1004B000892B09F467C11092B7001092B600CA01E7
:1004C0000C979093B5008093B4009093AA0080930A
:1004D000A90010928C0110928B011092A80010922A
:1004E000A70088E08093AB00DDC08091D700807FBB
:1004F000803609F047C19091DB0080E02091DC005C
:10050000BC01620F711D8091A7009091A800861711
:10051000970708F437C1EB01A896D093A800C093C1
:10052000A7001091DD00113151F4CA01849762E6F1
:1005300070E040E150E0B0D8009709F442C0E0918B
:100540008E00F0918F00608171818FEE90E040E12C
:1005500050E0A2D8009709F015C1113191F11A337A
:1005600009F010C127ED30E08091FF00803809F0DC
:1005700009C181E88093FF00D9015896F9013896A6
:1005800080E101900D928150E1F7E0918E00F091B1
:100590008F00AFEDB0E020813181C901FC0180E125
:1005A00001900D928150E1F7109202011092010129
:1005B0008AE300DF8095909590930201809301017A
:1005C000E5C0E097D093A800C093A70087E091E032
:1005D0009093B5008093B40080910501909106013D
:1005E000892B31F081E1E6DE8F5F9F4F09F0CAC0B1
:1005F00089EE91E09093AF008093AE0035C02889DA
:1006000039892115310559F180910101909102013B
:100610008217930721F52A893B892115310539F085
:100620008091FF009091000182179307C1F4CE01E1
:1006300062E770E040E150E02FD80097F1F0CE0182
:1006400062E670E040E150E027D80097B1F08FED0E
:1006500090E0BE0140E150E01FD8009771F067972D
:10066000D093AF00C093AE00C091AE00D091AF0068
:1006700081E0CD38D80718F685C01092B7001092E7
:10068000B60082E08093AB0087E091E09093B500E4
:100690008093B4009093AA008093A90010928C01DB
:1006A00010928B01C4DD20918B0130918C012115BA
:1006B000310509F467C0C901C0969093A8008093E2
:1006C000A700285F3F4F3093DB0088528093DC0007
:1006D00080E48093DE0081E18093DD0030930301AC
:1006E000209304011092060110920501E091AE00E2
:1006F000F091AF0080899189909300018093FF0071
:10070000828993899093020180930101E0918E0088
:10071000F0918F00AFEDB0E020813181C901FC0183
:1007200080E101900D928150E1F7AFEEB0E0809151
:10073000AE009091AF009C01F90180E101900D9213
:100740008150E1F787E091E09093B5008093B40089
:1007500081E130DE809590959093060180930501AC
:10076000892B31F48FEF9FEF909306018093050161
:1007700080E68093D7001092D8001092DA00109291
:10078000D90004C01092A8001092A7001092AB00EC
:10079000DF91CF911F9108950F931F93CF93DF9314
:1007A0008C018091AC009091AD0001969093AD00CA
:1007B0008093AC0080509D4730F080E090E19093B2
:1007C000AD008093AC0010929A0020E0A7E1B0E069
:1007D0001CC0322F3F5F822F90E08A9FF0018B9FD9
:1007E000F00D9A9FF00D1124E357FE4F80899189F7
:1007F000892B51F420939A0087E1289FD00111247E
:10080000A357BE4F49F43FC0232F253010F3209348
:100810009A00A0E0B0E037C09091AC008091AD00AC
:1008200050968C93509751969C93519753967C93E6
:100830006E9352970115110531F480E1ED01199283
:100840008A95E9F707C0ED01F80180E1019009926E
:100850008150E1F755965C934E93549780918E00AA
:1008600090918F0082589040959587952BEA3AEAAF
:10087000AC01429FC001439F900D529F900D1124E7
:1008800056968C935697CD01DF91CF911F910F9182
:100890000895282F86E0289FC00111248E579F4F6E
:1008A00090938F0080938E00222331F0213029F421
:1008B0008091A7001ED401C023D280E008951F9329
:1008C000CF93DF93CFEED0E010E0CE0160E872E08E
:1008D0004091C40297DD882381F4CE0165E472E083
:1008E000409144028FDD882311F081E007C0C9EBFD
:1008F000D0E01F3F11F01FEFE8CF80E0DF91CF91F4
:100900001F9108951F93182F8FEE90E060E872E01A
:1009100040E150E0C1D6009719F482E890E00BC0A6
:100920008FEE90E065E472E040E150E0B5D60097CC
:1009300049F488E890E090938F0080938E0081E0E6
:100940009FDD1AC0BCDF282F181791F08091DE00C0
:1009500081508093DE00882359F08091A700909108
:10096000A8000E979093A8008093A700822F91DF94
:100970001092A8001092A7001F910895DF93CF93C3
:10098000CDB7DEB760970FB6F894DEBF0FBECDBF10
:1009900080E291E09A83898386E098EF9C838B8341
:1009A00082E199E09E838D8380E093E298878F8334
:1009B0001A86198680E091E09C878B878FEF90E004
:1009C0009E878D878EEE91E0988B8F87E0918E00C9
:1009D000F0918F0020813181C901DC01FE01319647
:1009E00080E101900D928150E1F7E0918E00F0914D
:1009F0008F000280F381E02D88E6808360960FB639
:100A0000F894DEBF0FBECDBFCF91DF91089580E097
:100A1000089586D181B38F7581BB82B38F7582BBF8
:100A200083E084BB8D9A20E040E65AEECA0101972C
:100A3000F1F7A8952F5F2431C9F78D9820D008953C
:100A400025D0E7D10895809155028B3009F44FD11C
:100A500008959C01809155028A3011F081E008953B
:100A6000C901A7D10895FC018181809355028A5064
:100A7000823010F080E00895CF011CD1089585B731
:100A8000846085BF8BB780688BBF08951F93CF9319
:100A9000DF9360916602635067FD9DC080916302A1
:100AA000CCE0D0E0C81BD109C659DD4F809162026D
:100AB0008D3209F07EC0683009F08BC083EC8093E2
:100AC00056028AE58093900010929B008881807680
:100AD00039F0CE01C8DF282F8F3F09F459C05FC01D
:100AE0009A8110925F028981882321F4109260021A
:100AF00022E047C0853019F49093670241C08630E8
:100B000081F58B81813019F484E590E01FC082303B
:100B100019F486E690E01AC08330F1F4992341F489
:100B200086E290E0909365028093640224E015C011
:100B3000913041F48AE290E09093650280936402E0
:100B400028E10BC0923041F482E490E0909365027A
:100B50008093640222E101C020E080E480939B0046
:100B60001EC0883021F421E089E692E00CC0893073
:100B700019F49093690204C08A3011F421E001C095
:100B800020E08FE592E0909365028093640207C0B5
:100B9000888187FD2E8180E880939B0006C08F812D
:100BA000882319F48E81821708F0822F8093910098
:100BB00010C080919B0087FF0CC0CE014ADF8F3FA1
:100BC00021F48EE18093900004C0882311F01092EC
:100BD0009100109266028091900084FF5DC0809128
:100BE00091008F3F09F458C0182F893008F018E0A1
:100BF000811B809391008091560298E88927809309
:100C00005602112381F180919B0087FF06C087E582
:100C100092E0612FFCDE182F26C0209164023091F3
:100C2000650286FF0DC0A7E5B2E080E090E0F90123
:100C3000E80FF91FE491ED9301961817C1F708C06A
:100C4000912FD901E7E5F2E08D9181939150E1F781
:100C50001150812F90E01F5F0196820F931F909398
:100C600065028093640280919100882309F4EBDE91
:100C7000193060F487E592E0612F0AD1612F6C5F33
:100C80006C3041F08FEF8093910004C08FEF809320
:100C900091006EE1609390009AE080B3887231F425
:100CA0009150D9F71092670210926102DF91CF91B3
:100CB0001F910895FC0181818A3061F410929D009A
:100CC00010929C008281938190939F0080939E005C
:100CD0008FEF08958091C502882341F087ED90E061
:100CE000909365028093640280919E0008958091A4
:100CF000C502882311F41092B8001092C50208951D
:100D000081E08093C50210929D0010929C0080911A
:100D1000A7009091A80090939F0080939E00089553
:100D2000DF93CF93CDB7DEB760970FB6F894DEBFF1
:100D30000FBECDBF82E890E090938F0080938E002D
:100D400080E291E09A83898386E098EF9C838B838D
:100D500082E199E09E838D8380E092E298878F8381
:100D60001A8619861C861B861E861D8680E092E0E8
:100D7000988B8F872091820030918300C901DC011C
:100D8000FE01319680E101900D928150E1F7E091F2
:100D90008E00F0918F000280F381E02D80E480834B
:100DA00060960FB6F894DEBF0FBECDBFCF91DF9136
:100DB0000895CF93DF93482F792FC62FD0E020914D
:100DC0009C0030919D00225F3F4FC9018C0F9D1FF9
:100DD000803C910538F427533F4FC901642F4C2FB5
:100DE00050E067D480919C0090919D008C0F9D1FD6
:100DF00090939D0080939C0040E020919E00309154
:100E00009F008217930708F041E0842FDF91CF9174
:100E1000089520919E0030919F002115310511F118
:100E200080919C0090919D0082179307D8F0225FDB
:100E30003F4F3093A8002093A70010929F0010927C
:100E40009E0080E05FDD8091A7009091A800892B33
:100E500039F48091C502882329F41092B8000895CE
:100E60002EDD17DD0895A82FB92F80E090E041E036
:100E700050EA60956F5F58F42D9138EF822797956F
:100E8000879510F0842795273F5FC8F3F3CF089527
:100E9000EADF8D939D930895CF93CFB7CF93DF93E0
:100EA000859BFECF859B0BC0859B09C0859B07C09A
:100EB000859B05C0859B03C0859B01C089C06F933E
:100EC000C0916302DD27C659DD4F2F9365E5859BF1
:100ED00003C02F916F91E6CF0F931F934F9320E0A4
:100EE00040E15F9300B3087205FB27F93F9350E0A0
:100EF0003BE039C0187240642F77012F53501EC059
:100F0000406810B318722F7753501FC0406400B36D
:100F10002F770872D1F15350000023C0406210B304
:100F20002F77187291F15350000025C008721027D6
:100F3000515012F45D5F0000115027952C3F10B303
:100F4000C8F618720127015027952C3FC8F6422792
:100F5000499300B3087210274F73115027952C3F07
:100F6000A8F64695469510B3187279F001270150FE
:100F700027952C3F98F66B5A60F3315000B3B0F6CA
:100F800000C010E81ABF002717C03B503195C31BA3
:100F9000D04010E81ABF0881033CF9F00B34E9F0A7
:100FA000209161021981110F1213EDCF093651F111
:100FB0000D3211F0013E39F7009368023F915F91C5
:100FC0004F911F910F912F916F91CAB7C7FD68CFB5
:100FD000DF91CF91CFBFCF91189500916802002388
:100FE00069F310916602112339F534303AF13093E8
:100FF000660200936202109163023BE0311B309362
:1010000063021CC0009166020130B4F40AE530911D
:10101000900034FD14C000939000C6E5D2E013C0E8
:10102000052710E000C0000002BB1AC0052710E031
:10103000221F1DC010E021C04AE502C032ED432F3F
:10104000C4E1D0E032E011B31862959A02B311BB4B
:1010500058E220E865E320FF052702BB2795179596
:101060001C3FF0F66695B8F7B1F720FF052702BBE5
:10107000279517951C3FD0F62795179517FF05273D
:1010800000001C3F02BBB0F629913A9519F7077D85
:1010900010916702110FC651D04002BB11F010939E
:1010A000610210E81ABF006211B3177D402F477D1F
:1010B00054E05A95F1F702BB11BB42BB7FCF48D039
:1010C0008823B1F038D081E01DDC8091A700909199
:1010D000A800892B39F48091C502882349F4109225
:1010E000B8000895ECDBD5DB1092A8001092A700A1
:1010F0000895982F8091A4008823E1F48091A500A1
:101100008823C1F48091A1008823A1F41092A30048
:101110009093A4009FB7F89483E08093A10088E4A3
:101120008AB9929A5E9A9FBF80E38093A2008CE571
:101130008CB9969A08958091A400882341F4109266
:10114000A5009FB7F89480E98AB992989FBF089547
:101150008091A500882311F08091A50008959FB784
:10116000F89410BC83E389B986E880BD8AB18869A8
:101170008AB959989FBF8A9A8F9A8E9A1092A40022
:101180001092A5001092A3008091A400882341F43E
:101190001092A5009FB7F89480E98AB992989FBFF2
:1011A00008958091A1008823C9F081508093A10007
:1011B0008823A1F48091A400882381F09FB7F8943C
:1011C00083E08093A10088E48AB9929A5E9A9FBFD7
:1011D00080E38093A2008CE58CB9969A08951F92C3
:1011E0000F920FB60F9211248F939F93EF93FF935B
:1011F0008091A200882321F08CB91092A2004DC0EA
:101200008091A400882341F19091A3008091A400D3
:10121000981710F5E091A300F0E0E952FF4F90819C
:101220009C3551F4E091A300F0E0E952FF4F80813A
:101230008093A2009CB907C0E091A300F0E0E952BE
:10124000FF4F80818CB98091A3008F5F8093A300B2
:1012500083E08093A10021C08091A400882371F0D5
:101260001092A4008091C502882311F41092B80056
:1012700081E38093A2008CE58CB90FC01092A1008D
:1012800096988091A400882341F41092A5009FB7FE
:10129000F89480E98AB992989FBFFF91EF919F914E
:1012A0008F910F900FBE0F901F9018951F920F9265
:1012B0000FB60F9211248F939F93EF93FF935B9937
:1012C00002C05C9B02C08CB156C09CB18091A5004D
:1012D000882309F050C08091A400882309F04BC0F6
:1012E0008091A000882371F11092A000903309F43E
:1012F00042C0913321F58091A100882349F08FB736
:10130000F8941AB88FBF97988091A3008093A50096
:101310001092A1008091A400882369F19FB7F894EE
:1013200083E08093A10088E48AB9929A5E9A9FBF75
:1013300080E38093A2008CE58CB9969A1CC09C3502
:10134000D1F406C09C3521F481E08093A00013C045
:101350008091A300823B78F48091A100882359F00A
:10136000E091A300F0E0E952FF4F90838091A30049
:101370008F5F8093A300FF91EF919F918F910F90CA
:101380000FBE0F901F9018958091A60082608093E9
:10139000A60080E18093AB0080E090E008956F921A
:1013A0007F928F929F92BF92CF92DF92EF92FF92A5
:1013B0000F931F93CF93DF938C016B013A01FC01D4
:1013C00001900020E9F73197E81BF90B339718F4E7
:1013D00020E030E04BC0BB248B2C9924F401EE0FAD
:1013E000FF1FEE0FFF1FE957FF4FC591D4912097C4
:1013F00029F1CE0148D17C01C801BE01A7012DD140
:10140000892B69F4F401EE0FFF1FEE0FFF1FE75762
:10141000FF4F259134912115310519F40FC0B39474
:10142000DBCFC8018E0D9F1DB601A301F9010995FF
:101430009C018FEF2F3F380779F402C02FEF3FEF69
:10144000C114D10449F0C60163E970E04CE050E0FA
:1014500011D12CE030E00AC02115310539F48FE4B8
:10146000F60180838BE4818322E030E0C901DF91C3
:10147000CF911F910F91FF90EF90DF90CF90BF9091
:101480009F908F907F906F900895FC01DB01808189
:10149000882331F101C0319680818032E1F38823C5
:1014A000F9F01C920DC09C919295907F9C932081A5
:1014B000822F80538A3008F08750892B8C93319685
:1014C0009081892F80538A3070F3892F992787FD67
:1014D00090958F7D907081549040069720F302C0C4
:1014E000E0E0F0E0CF010895BF92CF92DF92EF925B
:1014F000FF920F931F93DF93CF9300D0CDB7DEB74A
:10150000FC016B018FEF8A8301C0319680818032AC
:10151000E1F3873629F0833709F090C0BB2404C07B
:10152000BB24B39401C0319680818032E1F7819170
:101530008032E9F38081992787FD90958F7D9070A7
:101540008934910549F08F34910541F08434910537
:1015500009F074C011E003C010E001C012E0319640
:1015600080818032E1F3992787FD90958F7D90707F
:101570008E349105A4F7CF01BE016F5F7F4F85DFE9
:10158000009709F45BC0F98021E0F21639F0F216F9
:1015900040F042E0F41609F051C008C023E330E007
:1015A00002C026E330E0EE24EA9404C020E330E0F9
:1015B00043E1E42EF901E10FF11D8F01BB2029F178
:1015C0001081C6016FE970E04AE050E053D0F0E3CB
:1015D000FF0EF601F582812F82958F708A3010F40C
:1015E000805D01C0895CF6018287812F90E08F7059
:1015F0009070212F2F700A9714F4205D01C0295C90
:10160000F60123872CE030E01BC0BE016F5F7F4FE7
:101610003CDF009799F0BE016E5F7F4F36DFF80127
:1016200020819A818E2D892380958223298192237E
:101630009E21892B808320E030E002C02FEF3FEF16
:10164000C9010F900F90CF91DF911F910F91FF90E3
:10165000EF90DF90CF90BF900895FB01DC0104C0B4
:101660008D910590801921F441505040C8F7881B96
:10167000990B0895FB01DC0102C005900D924150C9
:101680005040D8F70895FC0105900020E9F78095B7
:1016900090958E0F9F1F0895FB01DC0104C08D9172
:1016A0000190801921F441505040C8F7881B990BD4
:1016B0000895FB01DC0102C001900D9241505040A1
:1016C000D8F70895AA1BBB1B51E107C0AA1FBB1F77
:1016D000A617B70710F0A61BB70B881F991F5A95BE
:1016E000A9F780959095BC01CD010895F894FFCF9E
:1016F000000EFFFFFFFFFFFFFFFFFFFFFFFFFFFFEA
:10170000FFFF0000000000000000000000000000DB
:1017100000008002C40290024502440210028200CE
:021720005AFF6E
:00000001FF
